:020000040000FA
:100000008316FF2390000F30850014309F0080304E
:10001000810083121230990009309F003B20850136
:100020008516191F11280630A200A20B1528191FCA
:100030001128043090008E0120088F0010140C103D
:10004000A1019B3081000B11191B21140B1D2428C9
:1000500021182B2811280C1C202885120516343055
:1000600090003B200C108F018E0110140C1C3628C0
:100070000512851611289F149F183C281E08A00001
:02008000080076
:02400E00E43F8D
:00000001FF
